S02000006F70656E62746C5F6F6C696D65785F73746D3332683130332E737265630F
S31508000000500B0020D12A0008E52A0008E52A000836
S31508000010E52A0008E52A0008E52A0008E52A000876
S31508000020E52A0008E52A0008E52A0008E52A000866
S31508000030E52A0008E52A0008E52A0008E52A000856
S31508000040E52A0008E52A0008E52A0008E52A000846
S31508000050E52A0008E52A0008E52A0008E52A000836
S31508000060E52A0008E52A0008E52A0008E52A000826
S31508000070E52A0008E52A0008E52A0008E52A000816
S31508000080E52A0008E52A0008E52A0008E52A000806
S31508000090E52A0008E52A0008E52A0008E52A0008F6
S315080000A0E52A0008E52A0008E52A0008E52A0008E6
S315080000B0E52A0008E52A0008E52A0008E52A0008D6
S315080000C0E52A0008E52A0008E52A0008E52A0008C6
S315080000D0E52A0008E52A0008E52A0008E52A0008B6
S315080000E0E52A0008E52A0008E52A0008E52A0008A6
S315080000F0E52A0008E52A0008E52A0008E52A000896
S31508000100E52A0008E52A0008E52A0008E52A000885
S31508000110E52A0008E52A0008E52A0008E52A000875
S31508000120E52A0008E52A0008E52A0008E52A000865
S31508000130E52A0008E52A0008E52A0008E52A000855
S31508000140E52A0008E52A0008E52A0008E52A000845
S3150800015080B580B2002806D1DFF8BC0B0068012103
S315080001600182002008E0DFF8640B00680068804719
S31508000170DFF8A40B00680A3002BD80B5DFF89C0BD7
S315080001804078DFF8941B0968C97888421AD3DFF8E3
S31508000190880B00688078002814D1DFF87C0B00688B
S315080001A0808800280ED1DFF8700B0068DFF8681B1E
S315080001B00968C9788172DFF8140B006840688047BF
S315080001C0002000E0022002BD80B580B2002806D1DA
S315080001D0DFF8440B006801210182002008E0DFF8FF
S315080001E0EC0A006880688047DFF82C0B00680C3042
S315080001F002BD80B5DFF8200B0068C178DFF8180B60
S3150800020000684079DFF8182B126892699047DFF882
S31508000210081B0968897A00292AD0C0B200280BD1A0
S31508000220DFF8F41A09680979002905D1DFF8E81A10
S3150800023009688978002901D002201AE0C0B200288E
S3150800024016D1DFF8880A0068C0688047DFF8C80A50
S315080002500068DFF8C41A09684979C172DFF8B80A74
S315080002600068DFF8B41A0968C9780173002000E04D
S31508000270022002BD80B580B2002806D1DFF8980AB0
S31508000280006802210182002032E0DFF8980A002186
S315080002900180DFF8840A006800787F21084231D19E
S315080002A0DFF8740A0068407A810608D5DFF8741A00
S315080002B0097851F00201DFF86C2A117007E0DFF8BF
S315080002C0641A097811F0FD01DFF8582A1170400602
S315080002D00FD5DFF8500A007850F00100DFF8441A0D
S315080002E00870DFF8E809006800698047DFF8340A13
S315080002F002BDDFF8300A007810F0FE00DFF8241A95
S315080003000870EEE7DFF8100A0068007810F07F0042
S31508000310012802D1DFF80C0AEAE7DFF8FC090068D1
S31508000320007810F07F0002282CD1DFF8EC0900686D
S31508000330417911F00F00090611D5C0B2DFF8E819A6
S3150800034051F8200010F030001028CAD1DFF8D4097F
S31508000350007850F00100DFF8CC190870C1E7C0B288
S31508000360DFF8C41951F8200010F44050B0F5805F4A
S31508000370B7D1DFF8B009007850F00100DFF8A4190A
S315080003800870AEE70020B3E710B5DFF88C090068FF
S31508000390007810F07F0000280BD1DFF87C09006890
S315080003A0407A10F0DF00DFF87019096848720020FB
S315080003B096E0022840F09380DFF85C0900684088E0
S315080003C0002805D1DFF8500900680079002801D017
S315080003D0022085E0DFF84409DFF83C190968497905
S315080003E031F080031C00DFF83029126852791206B2
S315080003F006D5DFF8342952F8242012F0300205E039
S31508000400DFF8242952F8242012F440520078834257
S3150800041007D2002A05D0DFF800090068807A00288C
S3150800042001D102205CE0080611D5DFF8FC0850F877
S31508000430240010F0300010284AD12000C0B200F085
S315080004404AFD30212000C0B200F0B5FC40E0DFF8DC
S31508000450D80850F8240010F44050B0F5805F37D122
S31508000460002C1DD1DFF8C40890F82C1089B22000A2
S31508000470C0B200F090FDDFF8B00850F824004BF643
S315080004808F71084090F4805090F40050DFF8981867
S3150800049040F4004050F0800080B241F8240017E094
S315080004A02000C0B200F0FEFCDFF87C0850F82400FB
S315080004B04BF68F71084090F4805090F40050DFF8A6
S315080004C0681840F4004050F0800080B241F82400DB
S315080004D0DFF8F807006840698047002000E002203E
S315080004E010BD80B5DFF830080068417931F080002A
S315080004F0DFF8242812685279120606D5DFF828286C
S3150800050052F8202012F0300205E0DFF81C2852F8D5
S31508000510202012F44052DFF804381B7898420DD296
S31508000520DFF8F4371B685B88002B07D1002A05D053
S31508000530DFF8E4271268927A002A01D102202CE01B
S31508000540090612D5DFF8E01751F8201048F6BF72F1
S31508000550114091F01001DFF8D02741F4004151F025
S31508000560800189B242F8201011E0DFF8BC1751F873
S3150800057020104BF68F72114091F48051DFF8A827AE
S3150800058041F4004151F0800189B242F82010DFF8A9
S315080005903C07006880698047002002BD80B5DFF807
S315080005A078070068407A50F02000DFF86C17096871
S315080005B04872DFF818070068C0698047002002BD46
S315080005C0DFF854271268528A80B2002807D1888833
S315080005D0801ADFF8441709680882002001E00868D5
S315080005E01018704770B5DFF83007006810F110046E
S315080005F02088A16800291AD0002818D0A588A84202
S3150800060000D20500280080B2A16888470600208825
S31508000610401B2080608828186080002000F0A1FC1C
S315080006202A0092B2010089B2300000F010FD20883D
S3150800063000280CD0DFF8F8064FF44051018000215D
S31508000640002000F09BFCDFF8EC06302101802088B2
S31508000650A188884205D3DFF8C00600680321017225
S315080006601DE02088002805D0DFF8AC0600680521C3
S31508000670017214E02088002811D1DFF89C06006872
S3150800068006210172DFF8B006006880B2DFF8AC1602
S31508000690002241F81020DFF89C063021018070BD49
S315080006A0F8B5DFF87406006810F110052888DFF839
S315080006B0681609680C7A00281FD1042C1DD1DFF8AA
S315080006C080060078012812D1DFF86C06006880B22F
S315080006D0DFF86816002241F81020DFF858063021A6
S315080006E001800424DFF858060021017004E007247D
S315080006F0DFF84006102101802BE0AE88864201D340
S31508000700042400E00224B04200D20600300080B281
S31508000710A96888470700002000F016FC320092B24C
S31508000720010089B2380000F079FC310089B2002056
S3150800073000F024FC2888801B288068883018688088
S31508000740DFF8F00530210180DFF8E4054FF4405169
S315080007500180DFF8C40500680472F1BD10B50220F7
S31508000760DFF8B41509684C78DFF8AC15096809781C
S315080007707F2211424ED1092C02D1FFF7FEFC69E017
S31508000780052C1BD1DFF890050068C078802811DA9F
S31508000790DFF884050068807800280BD1DFF8780533
S315080007A000688088002805D1DFF86C050068807A23
S315080007B0002801D008206FE000204BE0032C10D160
S315080007C0DFF854050068C078012808D1DFF8480525
S315080007D000688088002802D1FFF7E0FE3AE0022090
S315080007E038E0012C36D1DFF830050068C0780128DA
S315080007F00ED1DFF8240500688088002808D1DFF8C4
S3150800080018050068407A800602D5FFF7BDFD21E08D
S3150800081002201FE0DFF800150968097811F07F014A
S31508000820012904D10B2C15D1FFF7E3FC12E0DFF800
S31508000830E8140968097811F07F01022909D1012C09
S3150800084002D1FFF7A1FD05E0032C03D1FFF749FE0E
S3150800085000E00220C0B200280BD02000C0B2DFF8AA
S31508000860C014096849698847C0B2032801D109201C
S3150800087012E0C0B2002801D008200DE00620DFF8FB
S31508000880B814096889B2DFF8B424002342F8113095
S31508000890DFF8A01430220A80DFF87C140968087291
S315080008A010BD38B5DFF870040068407800240025CC
S315080008B0062824D1DFF86004006800787F21084202
S315080008C040F0C680DFF8500400688078C0B201287E
S315080008D004D1DFF84C040068C469B9E0C0B2022844
S315080008E004D1DFF83C040068046AB1E0C0B203280A
S315080008F040F0AE80DFF828040068446AA8E00028C3
S3150800090071D1DFF814140968498800296BD1DFF81A
S3150800091008140968C988022965D1DFF8FC13096833
S31508000920097900295FD1DFF8F003006800787F2194
S31508000930084208D1DFF8E00300688088002802D161
S31508000940DFF8004484E0DFF8D0030068007810F090
S315080009507F00012814D10021DFF8BC030068407924
S31508000960DFF8BC23126892699047002870D1DFF837
S31508000970A8030068807A00286AD0DFF8C84367E0D1
S31508000980DFF894030068007810F07F0002285FD132
S31508000990DFF884030068407910F00F00DFF8781359
S315080009A00968497911F07001DFF86C2312685279E9
S315080009B0120606D5DFF8702352F8202012F030020E
S315080009C005E0DFF8642352F8202012F44052DFF8DD
S315080009D04C331B7898423BD2002939D1002A37D0AC
S315080009E0DFF8604334E0082809D1DFF82C030068F3
S315080009F000787F2108422BD1DFF84C4328E00A28EB
S31508000A0026D1DFF814030068007810F07F0001286B
S31508000A101ED1C1480068807A002819D0BE480068EF
S31508000A204088002814D1BC480068007900280FD1F6
S31508000A30B9480068C08801280AD10021B64800686C
S31508000A404079B74A126892699047002800D1BF4C8E
S31508000A502000002814D0B04800684582AE480068D7
S31508000A6084610020A0470020AB490968098A4FF62F
S31508000A70FF72914213D1A84800680921017267E004
S31508000A80A54800684078A649096809698847C0B238
S31508000A900328E9D1A04800680921017258E0C0B2CC
S31508000AA0022804D09C480068008A002804D19A4885
S31508000AB00068082101724BE0974800680078000634
S31508000AC03ED595480068C088009000989249096804
S31508000AD0098A884204D2904800680099018225E074
S31508000AE08D480068008A8C490968C98888421DD2E1
S31508000AF089480068008A8A49096891F82C1089B2E1
S31508000B00884203D28E48002101700FE082480068AF
S31508000B10008A8349096891F82C1090FBF1F201FBD1
S31508000B201200002802D18648012101707A4800681F
S31508000B307B49096891F82C108182FFF7B1FD07E01F
S31508000B40754800680321017279484FF440510180C5
S31508000B5031BD38B501247848006880B27C4931F83F
S31508000B601000400000F1804515F5C0456A48006848
S31508000B70007A092826D068480068297801706D1C13
S31508000B8065480068297841706D1CA4B215EB4405C8
S31508000B902800851C008800F039FA5F4909684880F2
S31508000BA0A4B215EB44052800851C008800F02EFA2F
S31508000BB0594909688880A4B215EB44055648006867
S31508000BC02988C1805448006801210172524800688A
S31508000BD0C088002802D1FFF7C1FD01E0FFF761FEDA
S31508000BE000F055F832BD80B54B480068007A0228F7
S31508000BF001D0042805D1FFF753FD47480068007A5D
S31508000C001CE0062819D144480068407805280ED10A
S31508000C104148006800787F21084208D13E480068AC
S31508000C20C07800F055F829480068006A80473C48B3
S31508000C30006880688047082000E00820364909686F
S31508000C40087200F024F802BD80B533480068007ABF
S31508000C50022801D0042801D1082012E0032801D077
S31508000C60052805D1FFF7BEFC2B480068007A08E086
S31508000C70072805D12A480068C0688047082000E090
S31508000C80082025490968087200F001F802BD80B5F8
S31508000C90264890F82C1089B2002000F07CF91E48EE
S31508000CA00068007A082806D121484FF4805101804F
S31508000CB020481021018018480068007A092801D1C7
S31508000CC0012000E00020C0B202BD00003407002069
S31508000CD030B412490A78002114E00B00DBB2124C3A
S31508000CE054F8233048F68F7423400C00E4B22343AB
S31508000CF043F4004353F080030C00E4B20A4D45F870
S31508000D002430491C9142E8D3C0B250F08000114902
S31508000D10086030BC704700002C070020E80000205F
S31508000D203007002028070020005C00400000002053
S31508000D303E07002040070020505C00400460004049
S31508000D40470700207502000851010008C90100087C
S31508000D50086000404C5C0040704710B450F8041B13
S31508000D6081B102681218001D50F8043BDC0744BF25
S31508000D70A9F10104E31852F8044B43F8044B091F80
S31508000D80F9D1EBE710BC70474FF6F8710840DFF869
S31508000D90641208607047C0B2DFF85C2252F820205F
S31508000DA048F68F131A40114389B2C0B2DFF84822B9
S31508000DB042F820107047C0B2DFF83C2252F82020D3
S31508000DC048F6BF731A40CB0601D592F01002890681
S31508000DD001D592F02002C0B2DFF81C1242F400429C
S31508000DE052F0800292B241F820207047C0B2DFF874
S31508000DF0082252F820204BF68F731A40CB0401D5EF
S31508000E0092F48052890401D592F40052C0B2DFF8F8
S31508000E10E81142F4004252F0800292B241F82020D2
S31508000E207047C0B2DFF8D01151F8201048F6BF72EB
S31508000E30114091F0100191F02001C0B2DFF8B821FD
S31508000E4041F4004151F0800189B242F82010704700
S31508000E50C0B2DFF8A41151F820104BF68F7211407A
S31508000E6091F4805191F40051C0B2DFF88C2141F41D
S31508000E70004151F0800189B242F820107047C0B293
S31508000E80DFF8741151F8201048F68F62114041F4CA
S31508000E90004151F0800189B2C0B2DFF85C2142F806
S31508000EA020107047C0B2DFF8501151F820104904DD
S31508000EB010D5C0B2DFF8401151F8201048F68F72ED
S31508000EC0114041F4404151F08001C0B2DFF82821B9
S31508000ED042F820107047C0B2DFF81C1151F82010F4
S31508000EE0490610D5C0B2DFF8101151F8201048F69F
S31508000EF08F72114041F4004151F0C001C0B2DFF8D1
S31508000F00F82042F820107047DFF8E820126892B2FD
S31508000F10C0B212EBC000DFF8E42089B2490889B2F2
S31508000F20490042F810107047DFF8C820126892B2DC
S31508000F30C0B212EBC000DFF8C82089B2490889B2EE
S31508000F40490042F810107047DFF8A810096889B2FE
S31508000F50C0B211EBC000DFF8A41051F8100080B23F
S31508000F607047DFF89010096889B2C0B211EBC0006B
S31508000F70DFF88C1051F8100080B27047DFF8742043
S31508000F80126892B2C0B212EBC000DFF8782089B2BC
S31508000F9042F810107047DFF85C20126892B2C0B2AF
S31508000FA012EBC000DFF8602012EB400089B23F293F
S31508000FB00BDB89B24A091F23194200D1521E92B28D
S31508000FC0910251F40041016007E089B24A08C90755
S31508000FD000D5521C92B29102016070470549096812
S31508000FE089B2C0B211EBC000074951F8100080055C
S31508000FF0800D7047505C0040005C00400060004077
S3150800100008600040046000400C600040010080B2A7
S31508001010C9B2090251EA102080B2704710B492B2E0
S31508001020521C521089B2490001F1804313F5C0439E
S3150800103009E00178401C047851EA042119809B1CB8
S315080010409B1C401C521E002AF3D110BC704792B25A
S31508001050521C521089B2490001F1804111F5C04174
S3150800106005E00B680380091D401C401C521E002A1F
S31508001070F7D17047DFF8FC045FF0FF310160DFF855
S31508001080F8045FF0FF310160704770B504000D0089
S315080010901600200000F00BFAFF2805D02819401E7C
S315080010A000F005FAFF2801D1002017E0600A4FF486
S315080010B000714843DFF8C4140968884207D12B0039
S315080010C032002100DFF8B00400F0F4F806E02B0047
S315080010D032002100DFF89C0400F0ECF870BD70B512
S315080010E004000D00200000F0E2F906002819401E51
S315080010F000F0DDF9F6B2FF2E02D0C0B2FF2801D10A
S31508001100002005E00100C9B23000C0B200F060F965
S3150800111070BD80B500200090DFF85C04006810F10F
S31508001120010F01D1012038E00098DFF84C14496816
S31508001130081800900098DFF840148968081800908D
S315080011400098DFF83414C968081800900098DFF88A
S3150800115028140969081800900098DFF81C144969D2
S31508001160081800900098DFF810148969081800908C
S315080011700098DFF80414C969081800900098C0435D
S3150800118000900098401C009000AA0421DFF8EC03A8
S31508001190006810F5A870FFF778FF02BD0020DFF899
S315080011A0DC13096809680818DFF8D0130968496864
S315080011B00818DFF8C813096889680818DFF8BC1327
S315080011C00968C9680818DFF8B413096809690818AE
S315080011D0DFF8A813096849690818DFF8A013096831
S315080011E089690818DFF89413096811F5A871096860
S315080011F00818002801D1012000E00020704780B5BA
S31508001200DFF87403006810F1010F07D0DFF86803F0
S3150800121000F093F8002801D100200EE0DFF854030F
S31508001220006810F1010F07D0DFF8480300F085F8D1
S31508001230002801D1002000E0012002BDDFF83C03B0
S315080012400068704780B54FF40072B1FBF2F303FBF8
S315080012501213002B01D000200BE002688A4201D14C
S31508001260012006E001604FF40072001D00F0ACF9A1
S31508001270012002BD38B504000D00BF48844208D1DC
S31508001280BC4C29002000FFF7DDFF002810D1002004
S315080012900FE0BA480068854203D1B74CB7480568DD
S315080012A0EFE7200000F049F80028EAD1002000E026
S315080012B0200032BD2DE9F04104000F0015001E0084
S315080012C0780A4FF4007101FB00F8206810F1010F4D
S315080012D007D141462000FFF7B5FF002801D10020BD
S315080012E029E02068404508D041462000FFF7C2FFA4
S315080012F00400002C01D100201DE02068381A0019CE
S31508001300071D00F073F9201D381AB0F5007F0AD3BF
S3150800131018F500712000FFF7ADFF0400002C01D17D
S31508001320002008E0271D287838707F1C6D1C761E63
S31508001330002EE6D10120BDE8F0812DE9F041040038
S315080013400125206800F0B3F8C0B2FF2801D10020BB
S315080013503CE000F09BF88A480068C00703D500F017
S315080013609FF8002032E08748006850F00100854960
S315080013700860002600E0761C802E1DD2206810EB3F
S31508001380860714EB8600D0F80480A7F8008001E0F1
S3150800139000F02CF97A480068C007F9D45FEA1840CB
S315080013A0788001E000F022F975480068C007F9D492
S315080013B038684045DFD0002572480068400840007C
S315080013C07049086000F06CF82800C0B2BDE8F081EA
S315080013D070B505000C00E4B2EDB2AC4201D20020B3
S315080013E053E06648007AEDB2854205D3634890F823
S315080013F09800E4B2A04201D2002046E000F046F888
S315080014005F480068C00703D500F04AF800203CE0B2
S315080014105C48006850F002005A4908602800C0B2CB
S3150800142000F06FF805002000C0B200F06AF8060068
S315080014302000C0B200F082F88019401E401B401CF4
S31508001440840A002606E000F0D1F84D480068C00777
S31508001450F9D4761CB6B2A4B2A6420DD2B6B24FF4EF
S31508001460806000FB0650484908604648006850F00E
S31508001470400044490860E8E74248006830F0020046
S315080014804049086000F00CF8012070BD3F4840490B
S3150800149001603E483F490160394834210160704780
S315080014A03848006850F0800036490860704738B5FB
S315080014B00400002500E06D1CEDB20D2D1FD200F0D2
S315080014C095F8EDB20C202D4900FB05100068844202
S315080014D0F1D3EDB20C20294900FB05100068EDB2E6
S315080014E00C21264A01FB0521496808188442E2D2E4
S315080014F0EDB20C20214900FB0510007A00E0FF2020
S3150800150032BD38B50400002500E06D1CEDB20D2D86
S3150800151011D200F06BF8EDB20C20184900FB05104B
S31508001520007AE4B2A042F0D1EDB20C20134900FBD8
S315080015300510006801E05FF0FF3032BD38B50400E1
S31508001540002500E06D1CEDB20D2D11D200F04EF80D
S31508001550EDB20C20094900FB0510007AE4B2A0425E
S31508001560F0D1EDB20C20054900FB0510406800E0FB
S31508001570002032BDF0000020F402002030280008C8
S315080015800C20024010200240142002400420024091
S3150800159023016745AB89EFCD80B500F034F8002804
S315080015A00DD000F069F800F0B5F800F030F80449FD
S315080015B008400449086000F02AF84068804701BDE1
S315080015C080FFFF1F08ED00E070B504000D0016004F
S315080015D005E0287820706D1C641C00F007F83000C0
S315080015E0461E80B20028F4D170BD7047704780B59A
S315080015F0FFF740FD01BD80B5FFF747FD02BD80B589
S31508001600FFF76DFD02BD80B5FFF7C8FD02BD80B5C9
S31508001610FFF714FE02BD80B5FFF77BFD002801D158
S31508001620002001E0FFF7EBFD02BD50F8041B61B195
S3150800163050F8042BD30744BFA9F101039A180023D5
S3150800164042F8043B091FFAD1EFE7704780B500F06E
S3150800165079F800F0B1FA25480221017001BD80B57C
S31508001660234800F002FB012805D120480221017019
S315080016701F4800F088F801BD80B500F0C2FA01BD28
S3150800168080B51A4A1278022A02D1C9B200F0BEFA07
S3150800169000F073F801BD15480078002805D0022827
S315080016A007D004D3032806D007E0002006E0002070
S315080016B004E03F2002E0002000E03F2080B27047AF
S315080016C00A480078002805D0022807D004D3032842
S315080016D006D007E0002006E0002004E03F2002E0F4
S315080016E0002000E03F2080B270470000EC00002098
S315080016F0CC05002080B500F00DF80D480D490160B5
S315080017000D48002101600D48052101600C480021A3
S31508001710016001BD0948002101607047074800685B
S31508001720C00304D506480068401C05490860704790
S3150800173014E000E03F19010018E000E010E000E0C6
S3150800174020070020DFF8500400210170DFF8480464
S3150800175000218164DFF84004002180F84210DFF898
S3150800176038040021A0F84410DFF82C040021817009
S31508001770DFF82404002141707047DFF81C040021BB
S3150800178080F84210704780B50178FF291ED100F015
S3150800179091F8DFF8040490F84200012802D11020DD
S315080017A000F07EF8DFF8F003B0F9440001280CDBFE
S315080017B0DFF8E403012180F84210DFF8DC03B0F912
S315080017C04410DFF8D80300F053F801BDDFF8C8135A
S315080017D0097801294BD10178C92932D0CC293FD0C3
S315080017E0CF293AD0D0292FD0D12933D0D2292ED0FB
S315080017F0F32917D0F4290FD0F5290AD0F6290ED0E7
S31508001800FA2912D0FC2913D0FD2914D0FE2915D0A7
S3150800181029E000F0D2F8BCE700F0F1F8B9E700F0EB
S31508001820C1F8B6E700F010F9B3E700F0A3F8B0E79F
S3150800183000F09AF8ADE700F07FF8AAE700F06DF837
S31508001840A7E700F035F9A4E700F054F9A1E700F09E
S3150800185012F99EE700F07FF99BE700F090F998E708
S3150800186000F0A4F995E7202000F01AF891E7ACE714
S3150800187080B589B2FFF704FF01BD10B4002302E06A
S315080018800478E318401C0C00611E002CF8D1DBB26A
S315080018901360012010BC7047BF4800214170704793
S315080018A0BD49FE22CA70BC490871BB480221A0F88E
S315080018B04410704710B50400FFF7EEFFB648012143
S315080018C00170B548FF21C170B34800210171B248C3
S315080018D0007950F01000B0490871AF4800214171F5
S315080018E0AD48AD4949794171FFF7D5FEAA498871D6
S315080018F0FFF7E6FEA849C871FFF7E2FE80B2000AC4
S31508001900A5490872A44801214172A34801218172A0
S31508001910A1480821A0F8441010BD10B504009E483F
S3150800192000210170FFF7B8FF9B48FF21C1709A4854
S315080019300121A0F8441010BD9749FF22CA709649A4
S3150800194000220A719449944A52784A7192490022AF
S315080019508A7191490022CA718F4900220A728E49FA
S315080019600622A1F84420704710B504000020FFF7AE
S3150800197097FF10BD8849FF22CA708749884A8A643A
S31508001980854900220A71844900224A718249002247
S315080019908A7181490722C1F807207F490822A1F8E0
S315080019A0442070477C49FF22CA707B494068886496
S315080019B079480121A0F84410704710B50400FFF7D4
S315080019C06AFE401E6178884203DA2220FFF768FF24
S315080019D014E0627892B27048816C7248FFF7F4FDA1
S315080019E06D48FF21C1706C48806C617808186A4997
S315080019F088646078401C6849A1F8440010BD10B599
S31508001A000400FFF748FE401E6178884203DA222068
S31508001A10FFF746FF17E0604861688164627892B212
S31508001A205D48816C5F48FFF7CFFD5B48FF21C170B9
S31508001A305948806C61780818574988646078401C52
S31508001A405549A1F8440010BD80B55349FF22CA7014
S31508001A50554A41685048806CFFF70FFF4E49087198
S31508001A604D48002141714C48002181714A4808219E
S31508001A70A0F8441001BD10B504004748FF21C17005
S31508001A80454800210171444800214171FFF703FED2
S31508001A904149887140480021C1713F4800210172BF
S31508001AA03D48002141723C480721A0F8441010BD6A
S31508001AB010B50400FFF7EFFD621C80B2411E3648E0
S31508001AC0806CFFF798FD002803D13120FFF7E8FE68
S31508001AD00FE03148FF21C170FFF7DDFD2E49896C03
S31508001AE080B2401E40182C4988642B480121A0F872
S31508001AF0441010BD10B50400FFF7CDFD801E6178B7
S31508001B00884203DA2220FFF7CBFE23E02248FF2192
S31508001B10C17021480121A0F844106078002807D137
S31508001B20FFF779FD002802D13120FFF7B9FE11E051
S31508001B30A21C61781848806CFFF75DFD002803D168
S31508001B403120FFF7ADFE05E01348806C6178081870
S31508001B501149886410BD80B541680F48806CFFF74D
S31508001B604EFD002803D13120FFF79AFE06E00A4809
S31508001B70FF21C17008480121A0F8441001BD10B525
S31508001B800400FFF709FD0448FF21C170024801213E
S31508001B90A0F8441010BD0000F8040020FB04002043
S31508001BA0002B0008FC040020FF04002080B531202B
S31508001BB0FFF776FE01BD000080B500F03AF9402136
S31508001BC0DFF8400400F048F9DFF83C1408704021BB
S31508001BD0DFF8380400F040F9DFF834140870DFF84D
S31508001BE028040078FF2804D0DFF824040078FF28AA
S31508001BF004D17E21DFF81C0400F02AFA00F034FA3A
S31508001C0001BD80B5002000F04FFA01BD70B5040093
S31508001C100D00EDB2402D04DB9E21DFF8F80300F03D
S31508001C2017FA2800C0B200F06FF8C0B2012804D035
S31508001C30A221DFF8E00300F00BFA00260EE0FFF71A
S31508001C40D5FCB6B2305D00F05FF8C0B2012804D00A
S31508001C50AB21DFF8C00300F0FBF9761C2800C0B200
S31508001C60B6B280B28642EAD370BD10B5040000F061
S31508001C706BFADFF8A4030078002814D1DFF89C0378
S31508001C8000F03AF801280CD1DFF890030078002814
S31508001C9007D0DFF8840301210170DFF884030021EF
S31508001CA00170002010BDDFF878030078DFF86C13A8
S31508001CB04018401C00F020F80128F2D1DFF8600334
S31508001CC00078401CDFF858130870DFF854030078D2
S31508001CD0DFF8481309788842E3D1DFF8440302782D
S31508001CE092B2DFF840132000FFF76EFCDFF82803F6
S31508001CF0002101700120D5E780B50100C4480078AD
S31508001D0000F01BF9C0B202BD80B50100C9B2BE48D9
S31508001D10007800F0BAF8C0B202BD38B5BA48007803
S31508001D2000F05EF90400E4B2002C2DD0E4B2412C98
S31508001D3000DB4024002512E000A9B348007800F033
S31508001D40FCF8C0B2012804D04FF4A771B14800F0DE
S31508001D507FF9EDB2B4489DF8001029546D1CEDB218
S31508001D60E4B2A542E8D3E4B2220092B24FF48071FD
S31508001D70AD48FFF753F9E4B2210089B20120FFF715
S31508001D80FDF80120FFF74DF831BD38B5A749012008
S31508001D9000F028FA040000250FE0ADB2A348295C3C
S31508001DA09B48007800F071F8C0B2012804D040F2D0
S31508001DB07311984800F04CF96D1CADB2A4B2A54257
S31508001DC0EBD30120FFF744F831BD30B400230024DB
S31508001DD023000BE0DBB2040F373401F8134000018F
S31508001DE0DBB211EB4304002565705B1CDBB2D2B293
S31508001DF0934208D2040F0A2CECD2DBB2040F30341B
S31508001E0001F81340EBE730BC704710B58848006806
S31508001E1088490C68884909680818002808D00822E3
S31508001E208649FFF7D2FF042285492000FFF7CDFF38
S31508001E3010BD8449844A002004E088744A61183138
S31508001E401832401CC0B20028F7D0887400204861B8
S31508001E507E487C490160704710B47C4A1268002AA3
S31508001E6001D1FF200FE0794A12685369774C236045
S31508001E7011749060D060002353741060C9B20818BA
S31508001E80401E5060907C10BC704738B504000D00A9
S31508001E90E4B2022C04DB40F2FD115E4800F0D8F8EB
S31508001EA0E4B21820674900FB0410407CE4B218210C
S31508001EB0644A01FB0421097C884201D100203BE0E9
S31508001EC0E4B218205F4900FB0410C0680570E4B24C
S31508001ED018205C4900FB0410407C401CE4B2182121
S31508001EE0584A01FB04214874E4B21820554900FBFE
S31508001EF00410C068401CE4B21821524A01FB0421B0
S31508001F00C860E4B218204F4900FB04104068E4B2E8
S31508001F1018214C4A01FB0421C96888420BD2E4B255
S31508001F201820484900FB0410E4B21821454A01FB71
S31508001F3004210968C160012032BD38B504000D00CE
S31508001F40E4B2022C04DB40F21F21324800F080F88C
S31508001F50E4B218203B4900FB0410407C002801D15C
S31508001F6000203CE0E4B21820364900FB04108068E3
S31508001F7000782870E4B21820324900FB0410407C2F
S31508001F80401EE4B218212F4A01FB04214874E4B22A
S31508001F9018202C4900FB04108068401CE4B2182164
S31508001FA0284A01FB04218860E4B21820254900FB71
S31508001FB004104068E4B21821224A01FB042189680A
S31508001FC088420BD2E4B218201E4900FB0410E4B282
S31508001FD018211C4A01FB042109688160012032BDD1
S31508001FE010B50400E4B2022C04DB40F23F21094894
S31508001FF000F02EF8E4B21820124900FB0410407CC9
S3150800200010BD000045050020440500208905002074
S315080020108805002064290008460700200C060020D1
S31508002020450700200D0600204C0600208C060020DF
S31508002030E8F7FF1FECF7FF1FF0F7FF1F7E000020F1
S315080020408E000020CC060020E4060020240700208D
S3150800205080B5034A106003480160FFF7C7FAFCE73A
S31508002060180700201C07002080B5094809490160A7
S3150800207007480068022101720748084901600848B4
S3150800208008490160044800680068804701BD00BF30
S315080020902C070020FC060020300700200000002046
S315080020A0340700205800002020490978002914D157
S315080020B01F49096851F010011D4A11601D49096838
S315080020C031F470411B4A11601A49096851F4E0411C
S315080020D0184A1160154901220A70C0B2012804D1B4
S315080020E015484FF40061016003E014484FF400619D
S315080020F0016070470E48006850F004000C490860FB
S315080021000F480068000900010D4908600C4800687E
S3150800211050F004000A49086070470A480068C0077A
S3150800212001D4012000E00020704700004407002089
S31508002130181002400410014014100140101001400C
S31508002140000801400808014080B517481749096882
S3150800215001801548008816490988084080050AD56F
S3150800216012484FF6FF51016012480078401C114989
S31508002170087000F055F80C4800880D490988084091
S31508002180000401D500F056F8074800880849098870
S315080021900840400506D505484FF6FF310160064858
S315080021A04068804701BD00BF42070020445C0040EC
S315080021B03C070020490700200000002006480021AF
S315080021C0016006484FF4064101800548034909881D
S315080021D00160002070470000445C00403C07002076
S315080021E0405C004070B504000D00002614F07F0026
S315080021F0FEF7F4FE060014F07F00FEF7B2FE32008A
S3150800220092B2010089B22800FEF721FF300070BDA6
S3150800221080B5FFF782FD01BD80B5FFF7B6FD01BDAC
S3150800222080B503480068052801D1FFF776FD01BD92
S315080022303807002080B50020ADF8000039E0864850
S315080022400078864951F82000ADF80000BDF8000076
S31508002250000414D580480078804951F8200040F6DB
S315080022608F7108407C4909787C4A42F821007A48EF
S3150800227000787B4911EB800050F8040C8047BDF8C4
S315080022800000000615D574480078744951F82000F6
S3150800229080B248F60F7108406F4909786F4A42F8CC
S315080022A021006D4800786F4911EB800050F8040C46
S315080022B080476D4800686D490880000440F1CA806F
S315080022C06A48008810F00F00634908706248007871
S315080022D00028B4D1664861490968018064480088C5
S315080022E010F03000634908806148008810F44050B7
S315080022F05F4908805948006880B24BF6BF710840AC
S3150800230090F4005090F0200080B240F4004050F065
S3150800231080005249086055480088C0062FD44F48A7
S31508002320006880B248F60F7108404C490860FEF70D
S315080023305AFC4A48006880B24BF6BF7108404C49BF
S315080023400988C90401D590F4805049490988890447
S3150800235001D590F4005047490988C90601D590F07F
S31508002360100044490988890601D590F0200080B2FA
S3150800237040F4004050F08000384908606AE0374869
S315080023800068ADF80000BDF8000000052ED53348FA
S31508002390006840F68F71084030490860FEF7D9FB9F
S315080023A02E48006880B24BF6BF710840304909884C
S315080023B0C90401D590F480502D490988890401D5AE
S315080023C090F400502B490988C90601D590F01000F1
S315080023D028490988890601D590F0200080B240F482
S315080023E0004050F080001D49086033E0BDF8000049
S315080023F000047FF55EAF1948006840F68F71084003
S3150800240016490860FEF720FC1448006880B24BF6AF
S31508002410BF71084016490988C90401D590F480504F
S3150800242013490988890401D590F40050114909888F
S31508002430C90601D590F010000E490988890601D50C
S3150800244090F0200080B240F4004050F0800003492C
S315080024500860FFE701BD000048070020005C004057
S31508002460B400002098000020445C00404207002089
S315080024703E0700204007002080B5FFF7C6FC5D48F0
S3150800248000680021817200F0D3F8FFF797FE5A48DA
S315080024900021016001BD80B556480068002181729F
S315080024A0544800685549C979417252480068002164
S315080024B0C1720020FEF768FC4FF400710020FEF799
S315080024C06AFC10210020FEF776FC40210020FEF76A
S315080024D02BFD80210020FEF717FD0020FEF7CFFC1C
S315080024E0474890F82C1089B20020FEF754FD0020CA
S315080024F0FEF7AEFC00210120FEF74DFC4FF480717B
S315080025000120FEF701FDC0210120FEF70DFD402147
S315080025100120FEF733FD40210120FEF73CFD4FF474
S3150800252040510120FEF762FC20210120FEF743FC02
S315080025300020FEF7CDFB30480121016001BD31487E
S31508002540807A002802D02C480521016070472A4865
S315080025500421016070477047704780B50021C0B2FA
S31508002560062812D123480068007810F07F00012859
S315080025700BD1204800684079002806D11D4800681C
S315080025808078212801D10FF261010800002801D1C5
S31508002590022009E017480068816116480068002291
S315080025A0428200208847002002BD0220704780B57D
S315080025B0154980B2FEF704F802BD80B5134980B20A
S315080025C0FDF7FEFF02BD80B50A490968C978C9B298
S315080025D0062901DB002006E0C9B20D4A12EBC1014B
S315080025E080B2FDF7EDFF02BD80B50A4980B2FDF75E
S315080025F0E7FF02BD2C07002038070020402A000804
S3150800260000000020FC060020D0000020D800002092
S3150800261030000020E0000020C9B2002901D00220C5
S3150800262005E0C0B2002801D0022000E00020704773
S3150800263080B50120FFF738FD01200B4980B20860FC
S315080026400A480021018008480849098801600848A5
S315080026500021016005484FF4E05101800248034912
S3150800266009880160002002BD405C00403C0700204C
S31508002670445C004080B500F005F800F0B5F800F0BD
S31508002680BFF8FCE700B583B0002000900020019059
S315080026904D48006850F001004B4908604B480068F7
S315080026A04B49084049490860474800684949084075
S315080026B0454908604448006830F48020424908606B
S315080026C04248006830F4FE004049086042485FF41A
S315080026D01F0101603C48006850F480303A490860A0
S315080026E03948006810F4003001900098401C0090AA
S315080026F00198002804D1009840F2DC518842EFD1B5
S3150800270031480068800303D469213448FFF7A0FCE8
S315080027103348006850F010003149086030480068B6
S31508002720800880002E4908602D48006850F0020095
S315080027302B4908602548254909680160234800682F
S3150800274050F40050214908602048006850F4806021
S315080027501E4908601D48006830F47C101B49086053
S315080027600920801E80041949096850F480300843FE
S31508002770164908601448006850F0807012490860CD
S31508002780114800688001FBD5104800688008800061
S315080027900E4908600D48006850F002000B490860B1
S315080027A00A48006810F00C000828F9D107480068A4
S315080027B030F48000054908600A48006850F40000B3
S315080027C00849086007BD00000010024004100240D6
S315080027D00000FFF8FFFFF6FE08100240CC280008AC
S315080027E0002002401C10024080B5FEF7FEFEFEF7F0
S315080027F081FFFEF7FCFEFEF729FF00F00BF801BD8E
S3150800280080B5FEF7F3FEFEF789FFFEF728FF00F016
S315080028100DF801BD80B5FFF76DFCFFF77EFC0028BB
S3150800282001D1FEF7B9FE00F001F801BD70470000BE
S315080028300060000800200000030000000080000877
S31508002840002000000400000000A00008002000008E
S315080028500500000000C00008002000000600000077
S3150800286000E0000800200000070000000000010842
S3150800287000200000080000000020010800200000D9
S315080028800900000000400108002000000A000000BE
S3150800289000600108002000000B000000008001080D
S315080028A0002000000C00000000A001080020000025
S315080028B00D00000000C00108002000000E00000006
S315080028C000E00108002000000F000000433A5C57B2
S315080028D06F726B5C736F6674776172655C4F706557
S315080028E06E424C545C5461726765745C44656D6FE6
S315080028F05C41524D434D335F53544D33325F4F6CF9
S31508002900696D65785F53544D3332483130335F49CA
S3150800291041525C426F6F745C6D61696E2E63000094
S31508002920433A5C576F726B5C736F66747761726556
S315080029305C4F70656E424C545C5461726765745C9A
S31508002940536F757263655C41524D434D335F535403
S315080029504D33325C4941525C766563746F72732EEF
S3150800296063000000433A5C576F726B5C736F667462
S31508002970776172655C4F70656E424C545C54617247
S315080029806765745C536F757263655C41524D434D60
S31508002990335F53544D33325C7573622E6300000007
S315080029A02C03570069006E005500530042002000B2
S315080029B0420075006C006B00200049006E00740030
S315080029C06500720066006100630065002603570013
S315080029D069006E0055005300420020004200750051
S315080029E06C006B00200044006500760069006300F7
S315080029F06500000010B5074979441831064C7C4437
S31508002A00163404E00A68081D511888470146A14291
S31508002A10F8D110BD08000000280000000FECFFFFE9
S31508002A205C060000F0000020000000002FE3FFFF16
S31508002A30F0000000D80000000000002000000000A0
S31508002A4009022000010100C0320904000002FF004B
S31508002A500004070581024000000705010240000046
S31508002A601A034F00700065006E0042004C005400C7
S31508002A7020005500730065007200000000F009F898
S31508002A80002801D0FFF7B6FF0020FFF7F3FD00F09E
S31508002A9002F80120704700F001B8000007463846E2
S31508002AA000F002F8FBE7000080B5C046C046024ABF
S31508002AB011001820ABBEFBE7260002001201100128
S31508002AC000000040501DAC60000101020301000037
S31508002AD0034B9D46C046C046C046C046FFF7CEFFDC
S31508002AE0500B002080B541210148FFF7B1FA01BD1E
S31508002AF020290008C046C046C046C046FFF7BEFFAC
S31508002B004F70656E424C540004030904792400088A
S31508002B109724000857250008592500085B25000852
S31508002B20AB25000819260008AF250008BB250008B4
S31508002B30C72500080000000040000000082B000818
S31508002B4004000000602A00081A000000CC290008CA
S31508002B50260000007C0000201C000000A0290008B8
S31508002B602C000000590D00083F250008590D0008E3
S31508002B70590D0008590D0008590D0008590D00088F
S31508002B80590D00084F2500081C0353004500520044
S31508002B903100320033003400350036003700380083
S31508002BA03900300011220008590D0008590D000897
S31508002BB0590D0008590D0008590D0008590D00084F
S31508002BC019220008590D0008590D0008590D00086A
S31508002BD0590D0008590D0008590D0008BC2A0008AF
S31508002BE012000000402A000820000000522A0008AF
S31108002BF0090000000301000004000000BA
S70508002AF5D3
